:100000004BEF0CF0FFFFFFFF00001200080E566ED2
:10001000FF0E556E562E01D003D0552EFED7FAD7BF
:100020001E0E556E552EFED71200100E556E552E13
:10003000FED7000012004950390807E3300E495C32
:1000400004E3010E4B6E26EF00F04B6A1200000134
:100050004B504F02F4CF54F0F3CF53F04C505002BA
:10006000F4CF56F0F3CF55F04B505002F3505426D6
:10007000F4505522E86A56224C504F02F350542651
:10008000F4505522E86A562250AE4BEF00F04B5028
:10009000555C4C5056584CAE52EF00F04F50555CEA
:1000A0005050565853C04BF054C04CF055C04DF012
:1000B00056C04EF012000001566A556A546A536ADF
:1000C000596A4E3453364F50535E5050D8A0503C6E
:1000D000545E5150D8A0513C555E5250D8A0523C6D
:1000E000565EE86AD8A0010E595E4E36070E576E6E
:1000F0004E34533654365536563659364F504EA038
:1001000095EF00F0535E5050D8A0503C545E5150D3
:10011000D8A0513C555E5250D8A0523C565EE86A79
:10012000D8A0010E595EA6EF00F053265050D8B06B
:10013000503C54265150D8B0513C55265250D8B05E
:10014000523C5626E86AD8B0010E59264E36572E34
:1001500078EF00F04D34533654365536563659360E
:100160004F504EA0C7EF00F0535E5050D8A0503C07
:10017000545E5150D8A0513C555E5250D8A0523CCC
:10018000565EE86AD8A0010E595ED8EF00F05326FB
:100190005050D8B0503C54265150D8B0513C552600
:1001A0005250D8B0523C5626E86AD8B0010E5926B3
:1001B0004D36070E576E4D34533654365536563637
:1001C00059364F504DA0F8EF00F0535E5050D8A074
:1001D000503C545E5150D8A0513C555E5250D8A06E
:1001E000523C565EE86AD8A0010E595E09EF01F054
:1001F00053265050D8B0503C54265150D8B0513CA2
:1002000055265250D8B0523C5626E86AD8B0010E56
:1002100059264D36572EDBEF00F04C34533654360A
:100220005536563659364F504DA02AEF01F0535EE1
:100230005050D8A0503C545E5150D8A0513C555E0F
:100240005250D8A0523C565EE86AD8A0010E595EC2
:100250003BEF01F053265050D8B0503C542651503B
:10026000D8B0513C55265250D8B0523C5626E86A78
:10027000D8B0010E59264C36070E576E4C34533603
:1002800054365536563659364F504CA05BEF01F078
:10029000535E5050D8A0503C545E5150D8A0513CB1
:1002A000555E5250D8A0523C565EE86AD8A0010E66
:1002B000595E6CEF01F053265050D8B0503C542694
:1002C0005150D8B0513C55265250D8B0523C5626C9
:1002D000E86AD8B0010E59264C36572E3EEF01F091
:1002E0004B34533654365536563659364F504CA04B
:1002F0008DEF01F0535E5050D8A0503C545E5150E9
:10030000D8A0513C555E5250D8A0523C565EE86A87
:10031000D8A0010E595E9EEF01F053265050D8B080
:10032000503C54265150D8B0513C55265250D8B06C
:10033000523C5626E86AD8B0010E59264B36070EB5
:10034000576E4B34533654365536563659364F5011
:100350004BA0BEEF01F0535E5050D8A0503C545E0D
:100360005150D8A0513C555E5250D8A0523C565ED8
:10037000E86AD8A0010E595ECFEF01F05326505025
:10038000D8B0503C54265150D8B0513C552652500C
:10039000D8B0523C5626E86AD8B0010E59264B36E2
:1003A000572EA1EF01F04BB0E4EF01F04F50532670
:1003B0005050D8B0503C54265150D8B0513C5526DE
:1003C0005250D8B0523C562612000150021000E0A4
:1003D00001C0E9FF02C0EAFF495200E0EF96EF9E3C
:1003E000EF9CEF9AEF98EF9449BEEF8E49BCEF8CEB
:1003F00049BAEF8A49B8EF880050010A03E1EF9447
:1004000003EF02F0EF84EF8604EC00F0495200E0C5
:10041000EF96EF9EEF9CEF9AEF98EF9449B6EF8E30
:1004200049B4EF8C49B2EF8A49B0EF880050010A15
:1004300003E1EF941DEF02F0EF84EF8604EC00F08F
:10044000EF960050010A03E106EC00F002D015EC33
:1004500000F012000001656B666B676B686B829041
:10046000646B200E0001645D2AE265C050F066C036
:1004700051F067C052F068C053F05036509051367A
:100480005236533650C065F051C066F052C067F026
:1004900053C068F082844F6A82B24F2A4F50501086
:1004A000656F51C066F052C067F053C068F0000E2F
:1004B00066136713681382940001642BD2D782807D
:1004C000FF0E00016515506EFF0E6615516EFF0E92
:1004D0006715526E1F0E6815536E50C065F051C0FF
:1004E00066F052C067F053C068F0040E4F6E50C003
:1004F0004BF051C04CF052C04DF053C04EF04F5035
:1005000009E04E324D324C324B324E9E4EBC4E8E36
:10051000FF0FF6D74BC065F04CC066F04DC067F0DA
:100520004EC068F012000001220E576E536A546AE2
:10053000556A566A5706D8B4C0EF02F0D8905632C2
:100540005532543253324E324D324C324B32D8A0A7
:100550009AEF02F05706D8B4B8EF02F04F50532686
:100560005050542251505522525056229FEF02F0C3
:100570004F5053265050542251505522525056221B
:1005800012006E0E00016B6F6F0E6C6F6E0E6D6F52
:100590002D0E6E6F660E6F6F6C0E706F6F0E716F3B
:1005A000610E726F740E736F200E746F700E756F24
:1005B000720E766F690E776F6E0E786F740E796FAC
:1005C000660E7A6F7B6B280E7C6F6E0E7D6F750EDC
:1005D0007E6F6C0E7F6F6C0E806F290E816F826B49
:1005E0008A6B8B6B886B896B66C04BF067C04CF075
:1005F00068C04DF0010E00016627000E67236823D6
:100600004BC0F6FF4CC0F7FF4DC0F8FF0900F5CF17
:100610004BF04BC085F04B52D8B4C0EF0AF0855177
:10062000250A0BE064C0E1FF65C0E2FF85C0E6FF7C
:10063000644B652B8A4B8B2BD7D70001866B876B5E
:10064000886B896B28D000018887010E6627000E11
:10065000672368235ED000018881010E6627000EA3
:100660006723682356D000018883010E6627000E99
:10067000672368234ED000018987010E6627000E8C
:100680006723682346D000018885010E6627000E87
:10069000672368233ED066C0F6FF67C0F7FF68C0D7
:1006A000F8FF0900F5CF90F0000190512D0ACBE042
:1006B00066C0F6FF67C0F7FF68C0F8FF0900F5CF16
:1006C00090F09051200AC7E066C0F6FF67C0F7FFC0
:1006D00068C0F8FF0900F5CF90F090512B0AC3E0F5
:1006E00066C0F6FF67C0F7FF68C0F8FF0900F5CFE6
:1006F00090F09051230ABFE066C0F6FF67C0F7FF95
:1007000068C0F8FF0900F5CF90F09051300ABBE0C7
:1007100001D098D7000188B38891000188B78895E7
:1007200066C0F6FF67C0F7FF68C0F8FF0900F5CFA5
:100730004BF0000E4C6E4BC049F01BEC00F04B52DE
:1007400038E00001866B876B000186C04BF087C0E4
:100750004CF00A0E4F6E000E506E27EC00F066C093
:10076000F6FF67C0F7FF68C0F8FF0900F5CF90F00B
:1007700090514B24866F000E4C20876F300E865FA1
:10078000000E875B010E6627000E6723682366C094
:10079000F6FF67C0F7FF68C0F8FF0900F5CF4BF020
:1007A000000E4C6E4BC049F01BEC00F04B52CCE1FC
:1007B00036D066C0F6FF67C0F7FF68C0F8FF0900D3
:1007C000F5CF90F0000190512A0A29E169C0E9FFB4
:1007D0006AC0EAFFEECF4BF0EECF4CF04BC0E9FF22
:1007E0004CC0EAFFEECF86F0EECF87F069C0E9FF9C
:1007F0006AC0EAFFEECF4BF0EECF4CF0020E4B2674
:10080000000E4C2269C0E1FF6AC0E2FF4BC0E6FF68
:100810004CC0E6FF010E6627000E6723682366C002
:10082000F6FF67C0F7FF68C0F8FF0900F5CF90F04A
:10083000000190512E0A74E1010E6627000E672315
:10084000682366C0F6FF67C0F7FF68C0F8FF0900BD
:10085000F5CF90F090512A0A2AE169C0E9FF6AC0F9
:10086000EAFFEECF4BF0EECF4CF04BC0E9FF4CC0AF
:10087000EAFFEECF83F0EECF84F069C0E9FF6AC0F3
:10088000EAFFEECF4BF0EECF4CF0020E4B26000EFF
:100890004C2269C0E1FF6AC0E2FF4BC0E6FF4CC0DA
:1008A000E6FF010E6627000E6723682337D000019C
:1008B000836B846B66C0F6FF67C0F7FF68C0F8FF04
:1008C0000900F5CF4BF0000E4C6E4BC049F01BEC0D
:1008D00000F04B5223E083C04BF084C04CF00A0E72
:1008E0004F6E000E506E27EC00F066C0F6FF67C03A
:1008F000F7FF68C0F8FF0900F5CF90F090514B2446
:10090000836F000E4C20846F300E835F000E845B7B
:10091000010E6627000E67236823CCD7000103D0A1
:100920000001836B846B66C04BF067C04CF068C0FD
:100930004DF0010E00016627000E672368234BC0AF
:10094000F6FF4CC0F7FF4DC0F8FF0900F5CF85F06A
:10095000FED08AC04BF08BC04CF012000001888999
:10096000E2D76B0E00018C6F000E8D6F836B846B72
:100970002DD00001888D27D126D10001888B000160
:10098000888F21D169C0E9FF6AC0EAFFEECF4BF042
:10099000EECF4CF04BC0E9FF4CC0EAFFEECF8CF03D
:1009A000EECF8DF069C0E9FF6AC0EAFFEECF4BF0F1
:1009B000EECF4CF0020E4B26000E4C2269C0E1FF38
:1009C0006AC0E2FF4BC0E6FF4CC0E6FF000E00012C
:1009D0008D1902E1000E8C1905E17C0E00018C6F6F
:1009E000000E8D6F00018E6B8F6B00018E518C2578
:1009F000E96E8F518D21EA6EEECF4BF04B5203E042
:100A00008E4B8F2BF2D70001835184110AE08F5156
:100A1000845D02E18E51835D04E283C08EF084C068
:100A20008FF0000187518F5D02E186518E5D06E2F5
:100A300000018E51865F8F51875B03D00001866B6A
:100A4000876B000188B717D086C04BF087C04CF089
:100A5000010E0001865F000E875B4B504C100BE0CF
:100A600064C0E1FF65C0E2FF200EE66E644B652BBB
:100A70008A4B8B2BE9D78EC04BF08FC04CF0010E08
:100A800000018E5F000E8F5B4B504C1013E08CC04A
:100A9000E9FF8DC0EAFFEECF4BF064C0E1FF65C017
:100AA000E2FF4BC0E6FF644B652B8C4B8D2B8A4BD2
:100AB0008B2BE1D7000188A717D086C04BF087C0E9
:100AC0004CF0010E0001865F000E875B4B504C100E
:100AD0000BE064C0E1FF65C0E2FF200EE66E644BF0
:100AE000652B8A4B8B2BE9D77FD569C0E9FF6AC09C
:100AF000EAFFEECF4BF0EECF4CF04BC0E9FF4CC01D
:100B0000EAFFEECF85F069C0E9FF6AC0EAFFEECFE9
:100B10004BF0EECF4CF0020E4B26000E4C2269C07B
:100B2000E1FF6AC0E2FF4BC0E6FF4CC0E6FF850E66
:100B300000018C6F000E8D6F010E8E6F000E8F6F97
:100B400062D7C00E00018813000E89133CD000014B
:100B50008551000AD8B4FDD685516C0AD8B4FED6AA
:100B60008551450AD8B4FDD68551660AD8B4F9D660
:100B70008551650AD8B4F5D68551670AD8B4F1D63F
:100B800085516F0AD8B4F5D68551640AD8B4F4D625
:100B90008551690AD8B4F0D68551700AD8B4EDD61B
:100BA0008551580AD8B4E9D68551780AD8B4E7D621
:100BB0008551730AD8B4E6D68551630A96E085510B
:100BC000750ABFE0B4D7C00E00018815906F89C0C8
:100BD00091F0000E9117000E911902E1000E90198C
:100BE000D8A485D0000188A929D069C0E9FF6AC0CE
:100BF000EAFFEECF4BF0EECF4CF04BC0E9FF4CC01C
:100C0000EAFFEECF8CF0EECF8DF0EECF8EF0EECF90
:100C10008FF069C0E9FF6AC0EAFFEECF4BF0EECF7C
:100C20004CF0040E4B26000E4C2269C0E1FF6AC056
:100C3000E2FF4BC0E6FF4CC0E6FF2FD069C0E9FFE2
:100C40006AC0EAFFEECF4BF0EECF4CF04BC0E9FFAD
:100C50004CC0EAFFEECF8CF0EECF8DF0000E00011D
:100C60008DBFFF0E8E6F8F6F000E8DBFFF0E8E6FCC
:100C70008F6F69C0E9FF6AC0EAFFEECF4BF0EECF9D
:100C80004CF0020E4B26000E4C2269C0E1FF6AC0F8
:100C9000E2FF4BC0E6FF4CC0E6FF800E00018F195B
:100CA0004B6E800E4B5C08E1000E8E5D05E1000E80
:100CB0008D5D02E1000E8C5D19E2030E00018813C8
:100CC000000E89134B6A4C6A4D6A4E6A8C514B5E1A
:100CD0008D514C5A8E514D5A8F514E5A4BC08CF0FB
:100CE0004CC08DF04DC08EF04EC08FF057D000013B
:100CF00088A929D069C0E9FF6AC0EAFFEECF4BF0AE
:100D0000EECF4CF04BC0E9FF4CC0EAFFEECF8CF0C9
:100D1000EECF8DF0EECF8EF0EECF8FF069C0E9FF11
:100D20006AC0EAFFEECF4BF0EECF4CF0040E4B263C
:100D3000000E4C2269C0E1FF6AC0E2FF4BC0E6FF33
:100D40004CC0E6FF2BD069C0E9FF6AC0EAFFEECFD6
:100D50004BF0EECF4CF04BC0E9FF4CC0EAFFEECFBA
:100D60008CF0EECF8DF0000E00018E6F8F6F000EB5
:100D70008E6F8F6F69C0E9FF6AC0EAFFEECF4BF05C
:100D8000EECF4CF0020E4B26000E4C2269C0E1FF64
:100D90006AC0E2FF4BC0E6FF4CC0E6FF000E000158
:100DA000841902E1000E831911E1000E4B6E00015F
:100DB0008F1908E14B508E1905E14B508D1902E156
:100DC0008C51000A03E10001834B842BC00E00010B
:100DD00088154B6E4BC094F0C3D0010E0001856F97
:100DE000000185510A0A39E0020E4F6E85C04BF0B2
:100DF000000E4C6E4D6E4E6E4F5007E04B364B90D2
:100E00004C364D364E36FF0FF8D7740E4B26190E62
:100E10004C22000E4D224BC0F6FF4CC0F7FF4DC0D8
:100E2000F8FF0900F5CF90F00900F5CF91F0090027
:100E3000F5CF92F00900F5CF93F0000193518F5D4B
:100E400008E192518E5D05E191518D5D02E1905175
:100E50008C5D03E30001852BC3D792D0010E000106
:100E6000856F00018551080A39E0020E4F6E85C07A
:100E70004BF0000E4C6E4D6E4E6E4F5007E04B36F1
:100E80004B904C364D364E36FF0FF8D79C0E4B2606
:100E9000190E4C22000E4D224BC0F6FF4CC0F7FF3E
:100EA0004DC0F8FF0900F5CF90F00900F5CF91F0A3
:100EB0000900F5CF92F00900F5CF93F000019351AE
:100EC0008F5D08E192518E5D05E191518D5D02E1EA
:100ED00090518C5D03E30001852BC3D751D0010EE7
:100EE0000001856F000185510C0A39E0020E4F6E3A
:100EF00085C04BF0000E4C6E4D6E4E6E4F5007E0AD
:100F00004B364B904C364D364E36FF0FF8D7BC0E55
:100F10004B26190E4C22000E4D224BC0F6FF4CC042
:100F2000F7FF4DC0F8FF0900F5CF90F00900F5CFAD
:100F300091F00900F5CF92F00900F5CF93F0000190
:100F400093518F5D08E192518E5D05E191518D5D68
:100F500002E190518C5D03E30001852BC3D710D0D3
:100F600000019451000AD8B438D79451C00AD8B4BB
:100F700034D79451800AD8B471D79451400AAFE065
:100F8000800E4B6E800E000184194B5C02E1835190
:100F9000855D03E283C085F00FD0800E00018419C7
:100FA0004B6E800E4B5C02E18551835D05E285C08E
:100FB00083F0000E0001846F0001865187110FE05D
:100FC000030E88154B6E89C04CF0000E4C164B502A
:100FD0004C1005E0010E0001865F000E875B800E5D
:100FE000000184194B6E800E87194B5C02E186511B
:100FF000835D06E200018351865F8451875B03D0E5
:101000000001866B876BC40E00018815906F8951B3
:10101000080B916F9151080A02E1400E901909E105
:1010200000018651871104E0010E865F000E875B88
:1010300020D0C00E00018815906F8951080B916F68
:101040009151080A02E1800E901913E1800E4B6E57
:10105000800E000187194B5C02E18651020806E20E
:10106000020E0001865F000E875B03D00001866BD5
:10107000876B000188A574D088A31BD0010E88154A
:101080004B6E89C04CF0000E4C164B504C1003E0D8
:101090002D0E4B6E02D02B0E4B6E64C0E1FF65C06F
:1010A000E2FF4BC0E6FF0001644B652B8A4B8B2BA4
:1010B00040D0010E000188154B6E89C04CF0000E27
:1010C0004C164B504C100BE064C0E1FF65C0E2FFD2
:1010D000200EE66E644B652B8A4B8B2B2AD0C00EFC
:1010E00000018815906F8951080B916F9151080A82
:1010F00002E1800E90191DE164C0E1FF65C0E2FFCE
:10110000300EE66E0001644B652B8A4B8B2B88AB4F
:1011100003D0580E4B6E02D0780E4B6E64C0E1FFC8
:1011200065C0E2FF4BC0E6FF0001644B652B8A4BB4
:101130008B2B00018651871112E064C0E1FF65C06E
:10114000E2FF300EE66E0001644B652B8A4B8B2B61
:10115000010E865F000E875B86518711EEE18ED00F
:1011600000018651871114E088B712D064C0E1FFF6
:1011700065C0E2FF200EE66E0001644B652B8A4BD2
:101180008B2B010E865F000E875B86518711EEE187
:10119000000188A31BD0010E88154B6E89C04CF04E
:1011A000000E4C164B504C1003E02D0E4B6E02D02F
:1011B0002B0E4B6E64C0E1FF65C0E2FF4BC0E6FF43
:1011C0000001644B652B8A4B8B2B15D0010E00015F
:1011D00088154B6E89C04CF0000E4C164B504C10CD
:1011E0000AE064C0E1FF65C0E2FF200EE66E644BDA
:1011F000652B8A4B8B2BC00E00018815906F89518F
:10120000080B916F9151080A02E1400E90190CE110
:1012100064C0E1FF65C0E2FF300EE66E0001644B82
:10122000652B8A4B8B2B2AD0C00E00018815906F3E
:101230008951080B916F9151080A02E1800E9019B3
:101240001DE164C0E1FF65C0E2FF300EE66E000103
:10125000644B652B8A4B8B2B88AB03D0580E4B6E9F
:1012600002D0780E4B6E64C0E1FF65C0E2FF4BC058
:10127000E6FF0001644B652B8A4B8B2B800E4B6E77
:10128000800E000184194B5C02E18351855D0CE204
:1012900064C0E1FF65C0E2FF300EE66E0001644B02
:1012A000652B8A4B8B2BEAD783C04BF084C04CF064
:1012B000010E0001835F000E845B4B504C10D8B4CC
:1012C00041D1C00E88154B6E4BC090F021D1020E5B
:1012D0004F6E83C04BF084C04CF0000E000184BF01
:1012E000FF0E4D6E4E6E4F5007E04B364B904C3616
:1012F0004D364E36FF0FF8D7740E4B26190E4C2282
:10130000000E4D224BC0F6FF4CC0F7FF4DC0F8FF5A
:101310000900F5CF4FF00900F5CF50F00900F5CFE7
:1013200051F00900F5CF52F08CC04BF08DC04CF05D
:101330008EC04DF08FC04EF05BEC00F00A0E4F6E89
:10134000000E506E516E526E5BEC00F053C04BF0CD
:1013500054C04CF055C04DF056C04EF0300E4B24EA
:10136000856FE5D088AB4CD0020E4F6E83C04BF03A
:1013700084C04CF0000E84BFFF0E4D6E4E6E4F5079
:1013800007E04B364B904C364D364E36FF0FF8D7B4
:101390009C0E4B26190E4C22000E4D224BC0F6FF20
:1013A0004CC0F7FF4DC0F8FF0900F5CF4FF0090022
:1013B000F5CF50F00900F5CF51F00900F5CF52F00C
:1013C0008CC04BF08DC04CF08EC04DF08FC04EF0F5
:1013D0005BEC00F00F0E4B16000E4C164D164E1621
:1013E000EC0E4B26190E4C22000E4D224BC0F6FF80
:1013F0004CC0F7FF4DC0F8FF0900F5CF85F04BD08A
:10140000020E4F6E83C04BF084C04CF0000E84BFC0
:10141000FF0E4D6E4E6E4F5007E04B364B904C36E4
:101420004D364E36FF0FF8D79C0E4B26190E4C2228
:10143000000E4D224BC0F6FF4CC0F7FF4DC0F8FF29
:101440000900F5CF4FF00900F5CF50F00900F5CFB6
:1014500051F00900F5CF52F08CC04BF08DC04CF02C
:101460008EC04DF08FC04EF05BEC00F00F0E4B16AF
:10147000000E4C164D164E16FE0E4B26190E4C2223
:10148000000E4D224BC0F6FF4CC0F7FF4DC0F8FFD9
:101490000900F5CF85F04BD0020E4F6E83C04BF0A4
:1014A00084C04CF0000E84BFFF0E4D6E4E6E4F5048
:1014B00007E04B364B904C364D364E36FF0FF8D783
:1014C000BC0E4B26190E4C22000E4D224BC0F6FFCF
:1014D0004CC0F7FF4DC0F8FF0900F5CF4FF00900F1
:1014E000F5CF50F00900F5CF51F00900F5CF52F0DB
:1014F0008CC04BF08DC04CF08EC04DF08FC04EF0C4
:101500005BEC00F0070E4B14856F300E85270FD073
:101510009051000AD8B4DBD69051C00AD8B4D7D6BF
:101520009051800AD8B41ED79051400AB5E064C0EB
:10153000E1FF65C0E2FF85C0E6FF644B652B8A4B87
:101540008B2BB2D688A71AD0800E4B6E800E8719CF
:101550004B5C02E18651000811E264C0E1FF65C006
:10156000E2FF200EE66E644B652B8A4B8B2B010E3F
:10157000865F000E875B86518711EFE1F4EF02F082
:101580008AC04BF08BC04CF01200006A48C049F092
:10159000E5EC01F0010E006E12003EC001F03FC00C
:1015A00002F03EC0E1FF3FC0E2FFE66A3EC001F04C
:1015B0003FC002F0110EE126E76A120EE15E06EC72
:1015C00000F0E78AE788E78604EC00F0E79606EC8F
:1015D00000F0E78AE788E78604EC00F0E79615EC70
:1015E00000F015EC00F0E78AE788E78604EC00F0ED
:1015F000E79606EC00F0E78AE798E78604EC00F04F
:10160000E79615EC00F0E78AE798E78604EC00F02F
:10161000E796E78EE79CE78604EC00F0E79615EC8A
:1016200000F0000EE76EE78604EC00F0E796E78E28
:10163000E78CE78AE788E78604EC00F0E79615EC8C
:1016400000F0000EE76EE78604EC00F0E796E7880E
:10165000E78604EC00F0E79606EC00F0000EE76E7B
:10166000E78604EC00F0E796E78CE78AE78604EC6F
:1016700000F0E79615EC00F0010E006E12000FD09E
:10168000800E3E6E19D0C00E3E6E16D0940E3E6E89
:1016900013D0D40E3E6E10D0800E3E6E0DD03E5054
:1016A000010AEEE03E50020AEEE03E50030AEEE090
:1016B0003E50040AEEE0F0D73F044B6E3E504B26FE
:1016C0004BC03EF04BC049F0E5EC01F0006A426AC5
:1016D000436A42504024E96E43504120EA6EEECF07
:1016E0004BF04B520DE042504024E96E43504120F4
:1016F000EA6EEECF49F0E5EC01F0424A432AE9D721
:10170000010E006E120007C003F008C004F009C00B
:1017100005F00AC006F00BC007F00CC008F00DC0C1
:1017200009F00EC00AF00FC00BF010C00CF011C091
:101730000DF012C00EF013C00FF014C010F015C061
:1017400011F016C012F02AEC02F04BC013F04CC09E
:1017500014F04DC015F04EC016F00F504B2610502F
:101760004C2211504D2212504E220B504B260C5041
:101770004C220D504D220E504E2207504B26085041
:101780004C2209504D220A504E2203504B26045041
:101790004C2205504D2206504E22050E4F6E000E73
:1017A000506E516E526E5BEC00F0940E4F6E000E58
:1017B000506E516E526E93EC02F0640E4F6E000E3E
:1017C000506E516E526E5BEC00F01200430E000141
:1017D000626F000E636F3EC064F03FC065F040C0B2
:1017E00066F041C067F042C068F0620E696F000E9B
:1017F0006A6FC1EC02F04BC060F04CC061F04B501E
:101800003E24E16E4C503F20E26EE66A60C04BF031
:1018100061C04CF01200406A416A40503E24E96EBB
:1018200041503F20EA6EEECF4BF04B520DE040505E
:101830003E24E96E41503F20EA6EEECF48F0C5EC01
:101840000AF0404A412AE9D71200500E176E490E9D
:10185000186E430E196E500E1A6E720E1B6E6F0EBE
:101860001C6E6A0E1D6E650E1E6E630E1F6E740E6C
:10187000206E200E216E420E226E6F0E236E610EC0
:10188000246E720E256E640E266E276A170E286E61
:10189000000E296E120025EC0CF00E0EC16E936A3C
:1018A000FF0E826E020E946E810E3E6E0F0E3F6E24
:1018B000CDEC0AF0010E496EE5EC01F00C0E496E1C
:1018C000E5EC01F0010E3E6E010E3F6E28C040F0C7
:1018D00029C041F03FEC0BF04F6A82BE4F2A010E47
:1018E0004F184B6E000E4BB0800E8218800B821A80
:1018F00083EC0BF02A0E3E6E000E3F6E100E406E13
:101900001A0E416E000E426E4BC043F04CC044F0C4
:101910004DC045F04EC046F0E40E476EE6EC0BF0CD
:10192000C00E496EE5EC01F02A0E3E6E000E3F6ED1
:101930000BEC0CF0020E576EFF0E566EFF0E556E3E
:10194000572E01D007D0562E01D003D0552EFED7EA
:10195000FAD7F6D7060E566EFF0E556E562E01D0EC
:1019600003D0552EFED7FAD70A0E556E552EFED748
:10197000B3D7FFD7010000000A0000006400000098
:10198000E803000010270000A086010040420F007D
:101990008096980000E1F50500CA9A3B010000001E
:1019A0001000000000010000001000000000010015
:1019B0000000100000000001000000100100000005
:1019C00008000000400000000002000000100000BD
:1019D0000080000000000400000020000000000162
:1019E00000000008000000400000000030313233E9
:1019F00034353637383941424344454600FF3031AB
:101A0000323334353637383961626364656600FFD6
:101A10002530386C642078302E3125635600FFFF66
:020000040030CA
:0E000000FFF8FFFEFFFFBBFFFFFFFFFFFFFF4C
:00000001FF
